:1000000000308A0004280000FF238316900000308F
:100010008A005D2B820720342034203420342034A1
:10002000523461346C3465346E34743469347334EE
:1000300073346534753472345F34733465347234B8
:1000400076346F345F3431343234463436343734B6
:1000500035345F345634303432342D343234303425
:1000600000340034003400340034003400343330C1
:100070008400000803194B280130A100A001A00B47
:100080003F28A10B3E284A30A000A00B45280000C5
:100090000000800B3C288A2B0C30A1001F08C339BC
:1000A00021049F000330A000A00B54289F149F1828
:1000B00057281E08A700A70CA70C3F30A70504303F
:1000C000A1001F08C33921049F000330A000A00B2A
:1000D00067289F149F186A281E08A900A90CA90C5C
:1000E0003F30A90500342510A601A801AA0803196C
:1000F0007A2800304C208B2B90018F018E010C1040
:1001000085309000B401B501331000303318013050
:10011000003A031DD028003085190130013C031D31
:100120009E28340B9628B40A0F08B6003408033C06
:10013000031D9D28B40A0F08B800AA28B408031D9F
:10014000A3280130B4003408023C031DAA28B40AD5
:100150000F08B700003005190130013C031DBD2810
:10016000350BB528B50A0F08B9003508033C031D47
:10017000BC28B50A0F08BB00C928B508031DC22852
:100180000130B5003508023C031DC928B50A0F0827
:10019000BA0000300C180130013C031933148528D3
:1001A0009001B31033113408043C031DE328B31449
:1001B00036083802BC003C08393C0318E2283C08E9
:1001C000643C031CB310AA013508043C031DF42849
:1001D000331539083B02BC003C08393C0318F328AE
:1001E0003C08643C031C3311B31C1829331D182927
:1001F0003908360203180A2936083902BD003908C1
:1002000038023D02031807290330AA0009290430E7
:10021000AA00172939083602BD0036083B023D0204
:10022000031815290430AA0017290330AA00202931
:10023000B31C1C290130AA00331D20290230AA005A
:100240008C2B90018F018E010C100030851901302C
:10025000003A0319252985309000003085190130B6
:10026000013C03192D2990010F08A3000E08A000DE
:100270000F082302031D34292008AD002308AE0017
:10028000251000300C180130013C031925142E08EC
:10029000033C031C5129031D50292D081F3C031842
:1002A00025142E08083C03185C29FF3A031D5B291E
:1002B0002D08C43C031C25140034B601B5013508D3
:1002C0003F3C031C6D292708260203186929A60A4A
:1002D0006B29A601B60AB50A5F293608AB070318D1
:1002E000AC0A2E082C02031C8029031D7B292B0835
:1002F0002D02031880292E08AC002D08AB00A601A2
:100300000034B601B50135083F3C031C912927088C
:10031000260203188D29A60A8F29A601B60AB50A56
:1003200083293608AB020030031C0130AC022C08D4
:100330002E02031CA629031DA1292D082B02031838
:10034000A6292E08AC002D08AB00A60100342B080E
:10035000003CB500B6012C08031C2C0FB60201307E
:10036000B7000030031C0130B702B8010030031C95
:100370000130B80236088F0035088E000C10851643
:100380008530900000300C180130003A0319C22962
:100390008512003425102121003025180130003A43
:1003A000031D042A2D082B02B3002C08B4002E08CC
:1003B000031C2E0FB402B408031DE2293308073CC6
:1003C0000318032A3408FE3C0318ED29FF3A031DE5
:1003D000032A3308F83C031C032A2C082E02031CB2
:1003E000F929031DF7292D082B020318F9295D218E
:1003F000032A2E082C02031C032A031D022A2B08A1
:100400002D02031C8121A721A52B90018F018E01B4
:100410000C10003005190130003A0319092A853003
:100420009000003005190130013C0319112A900198
:100430000F08A3000E08A0000F082302031D182AAE
:100440002008B1002308B20000300C180130013C34
:10045000031925143208033C031C342A031D332AD4
:1004600031081F3C031825143208083C03183F2AA2
:10047000FF3A031D3E2A3108C43C031C25140034F6
:10048000B601B50135083F3C031C502A2908280253
:1004900003184C2AA80A4E2AA801B60AB50A422A0D
:1004A0003608AF070318B00A32083002031C632A6B
:1004B000031D5E2A2F0831020318632A3208B00098
:1004C0003108AF00A8010034B601B50135083F3C42
:1004D000031C742A290828020318702AA80A722A01
:1004E000A801B60AB50A662A3608AF020030031C16
:1004F0000130B00230083202031C892A031D842A0D
:1005000031082F020318892A3208B0003108AF00E1
:10051000A80100342F08003CB500B6013008031CC8
:10052000300FB6020130B7000030031C0130B702B3
:10053000B8010030031C0130B80236088F003508BE
:100540008E000C1005148530900000300C1801301E
:10055000003A0319A52A05100034251005220030A1
:1005600025180130003A031DE72A31082F02B30095
:100570003008B4003208031C320FB402B408031D63
:10058000C52A3308073C0318E62A3408FE3C031842
:10059000D02AFF3A031DE62A3308F83C031CE62A5A
:1005A00030083202031CDC2A031DDA2A31082F022C
:1005B0000318DC2A4022E62A32083002031CE62A0D
:1005C000031DE52A2F083102031C64228A22C12B55
:1005D00025102A08033C031DF02A21210522F22AB6
:1005E00005222121003025180130003A031D5C2B23
:1005F0002D082B02B3002C08B4002E08031C2E0F6C
:10060000B402B408031D082B3308073C0318292B38
:100610003408FE3C0318132BFF3A031D292B330823
:10062000F83C031C292B2C082E02031C1F2B031D36
:100630001D2B2D082B0203181F2B5D21292B2E08A3
:100640002C02031C292B031D282B2B082D02031C15
:10065000812131082F02B3003008B4003208031C96
:10066000320FB402B408031D392B3308073C0318BA
:100670005A2B3408FE3C0318442BFF3A031D5A2B17
:100680003308F83C031C5A2B30083202031C502B51
:10069000031D4E2B31082F020318502B40225A2BDA
:1006A00032083002031C5A2B031D592B2F0831022C
:1006B000031C6422A7218A22E62B84011F308305B4
:1006C00083161F08F0399F0083121F1307309F0005
:1006D000073099008316050803308312A000A00B91
:1006E0006F2B19088C1185013F30650083161F0898
:1006F000F0390A389F0083121F1383161F080F3921
:1007000030389F0083121F080C3901389F00C83011
:10071000B300372873287C2825102A0BA72B00301C
:1007200085190130013C03198F2B21210030251838
:100730000130013C031D9E2B8A0100281F306500FB
:100740002E08AC002D08AB00CA294C20A42B2A0887
:10075000023C031DC32B003005190130013C031975
:10076000AB2B0522003025180130013C031DBA2BAC
:100770008A0100283E3065003208B0003108AF0021
:10078000AD2A4C20C02B2A08033C0319CB2B2A0886
:10079000043C031DE82B003085190130013C03198E
:1007A000CB2B21210522003025180130013C031DEF
:1007B000DB2B8A0100281E3065002E08AC002D08B6
:1007C000AB003208B0003108AF00E82A4C20E52B1E
:0607D0008A01002863000D
:02400E00C439B3
:00000001FF
